:10000000FDC017C1F7C215C114C113C112C111C17E
:1000100083C30FC10EC10DC1CFC30BC10AC1B0CD87
:1000200091CDBDCDC7CDD1CDDECDFBCD76167B1725
:10003000811886198B1A911B961C9B1DA11EA61F49
:10004000AB20B121B622BB23C124C625CB26D127A4
:10005000D628DC29E12AE62BEC2CFF0B000000005F
:10006000A60EF9154C1DF22B3E498A6601020304C7
:10007000050607030303030414E6FF0000005AFF0C
:10008000FFFF000046FF1EFF000050FF1EFF0000A4
:1000900019FFFFFFFF00256E183F96FFFFFF0000CE
:1000A000000000468CFF146EFFFFFF0000000738C1
:1000B00089FF1E78FFFF0000000050FF1EFFFF00B9
:1000C000000050FF78FF000046FFFF0000FF00FF28
:1000D0000000000000000000000000000000000020
:1000E0000000000000000000000000000000000010
:1000F0000000000000000000000000000000000000
:1001000000000000000000000000000000000000EF
:1001100000020304050708090B0C0E0F1112141638
:1001200017191B1D1E20222426282A2C2F31333577
:10013000383A3C3F424447494C4F5255575A5D600C
:1001400064676A6D7174777B7E8286898D919599DB
:100150009DA1A5A9ADB2B6BABFC4C8CDD2D6DBE0C9
:10016000E5EAEFF4FAFF03030304040405050606B9
:100170000708090A0B0C0D0E0F11121416181A1C81
:100180001E212326292C2F33363A3E42464A4F530E
:10019000585D63686E747A80878E959CA4ACB4BCFD
:1001A000C4CDD6DFE9F3FDFFFFFFFFFFFFFFFFFF39
:1001B000FFFFFFFFFFFFFFFFFFFFFFFFFFFFFFFF4F
:1001C000FFFFFFFFFFFFFFFFFFFFFFFFFFFFFFFF3F
:1001D000FFFFFFFFFFFFFFFFFFFFFFFFFFFFFFFF2F
:1001E000FFFFFFFFFFFFFFFFFFFFFFFFFFFFFFFF1F
:1001F000FFFFFFFFFFFFFFFFFFFFFF0011241FBEF8
:10020000CFE5D2E0DEBFCDBF10E0A0E6B0E0E0E099
:10021000FDE102C005900D92AA39B107D9F720E09F
:10022000AAE9B0E001C01D92A43FB207E1F7D1D71F
:1002300065CDE6CE20ED37E0019720F0F90131974A
:10024000F1F7FACF08959091EC00992349F08823B3
:1002500021F083E187BBC49A089583E087BBC498EB
:100260000895815090E0FC01E053FF4F2491FC0180
:10027000EA59FE4F849189BD28BD8091E80088230A
:1002800011F080E0E0CF0895CF93DF93E091ED008F
:10029000F0E0E459FF4F84918093E2001092CE0089
:1002A0001092D8009091F200992341F09091F100C2
:1002B0009093D9001092CF0092E001C091E020E02D
:1002C00030E0482F50E0692F70E0241735072CF5F7
:1002D000A091ED00B0E0AA0FBB1FAC59BF4FED914C
:1002E000FC91E20FF31FE491E901C60FD71FDE0175
:1002F000A852BF4FEC93A091ED00B0E0AA0FBB1F36
:10030000A458BF4FED91FC91E20FF31FE491C2534B
:10031000DF4FE8832F5F3F4FD8CF890F8093E200F4
:10032000DF91CF910895811108C019BC18BC80914C
:10033000E800882319F081E086CF93CF089581E00B
:100340008093CD0093E09093F1008093CB0092E0F6
:100350009093E60095E09093ED008093F200109268
:10036000CC001092F0008093EF001092E300809395
:10037000EC000895CF93DF931F92CDB7DEB79FEFC8
:1003800098BD90E0698356DF18BC6981862F90E0A4
:100390000F90DF91CF914ECF8091CD008093B90027
:1003A0001092CD001092F3008BE58093BB0080E0AB
:1003B0004ACF8091B9008093CD001092C600809101
:1003C000CD00882319F01092BB0008958091BA00E7
:1003D0008093BB000895EF92FF920F931F93CF93EA
:1003E000DF93C82F8B017B01EE0CFF1CEE0CFF1C72
:1003F000D8E2CC2371F081E026DFD9BD18BCC8015A
:1004000019DF80E020DF19BC18BCC70113DFC15021
:10041000F0CFDF91CF911F910F91FF90EF90089552
:100420001F93CF93DF93C82FD62F18E2CC2301F16F
:100430008091BB008D131CC081E005DF8091EC0032
:10044000882321F08091E300811102C019BD18BCFE
:100450008AEF90E0EFDE80E0F6DE19BC18BC87E79B
:1004600091E0E8DE8091BB008D1302C0C150DECF69
:10047000DF91CF911F9108951F93CF93DF93D62FD4
:100480006AE001DC192F6D2FCBDFC091BB00CD13CB
:1004900010C080E293E0CEDE6C2F812FC1DF80910F
:1004A000BB008C1306C080ED97E0DF91CF911F91C8
:1004B000C1CEDF91CF911F910895EF92FF920F93DC
:1004C0001F93CF93863018F006E910E002C00AEFC0
:1004D00010E07801EE0CFF1CC82FCC23D1F019BC22
:1004E00018BCC801A7DE81E0AEDE8091CD00882374
:1004F00021F08091E50017DF06C08091CA0090913D
:10050000E40099BD88BDC70195DE80E09CDEC15046
:10051000E4CFCF911F910F91FF90EF900895EF924C
:10052000FF920F931F93CF938C017C01F594E79476
:10053000C62FCC2351F081E086DEC8017BDE80E04F
:1005400082DEC70177DEC150F4CFCF911F910F91AA
:10055000FF90EF900895CF93C82F68E270E082E09B
:100560003ADF80EF90E066DE64E670E08C2F33DFE8
:100570001092BC00CF91089586B383FB882780F941
:1005800091E098278091A400880F892B8093A40084
:100590009091A300992311F08F7001C08170809316
:1005A000A3008091A30090E008958091BB0080316A
:1005B00020F48091BB008093BA008091BB008F5FD4
:1005C0008093BB009091E200891710F01092BB005D
:1005D00008958091BB008093BA008091BB00811187
:1005E00003C08091E20002C08091BB0081508093E3
:1005F000BB00089518958EBB6DBB84E28CBB86E270
:100600008CBBE199FECF0895CF93DF932091BB007F
:100610008091ED009091CD00880F880F880F9795FD
:1006200099279795692F682B622B6093EE00209194
:10063000CC003091F0009091F1008091CB00330F0D
:10064000990F990F932B922B8295880F807E892B7F
:100650008093C9004091C8005091EC003091EF00A8
:100660009091E3008091F2007091E600550F330FF6
:10067000330F352B342B990F990F990F292F232BDB
:100680008295807F982F922B872F8295880F807E6E
:10069000892B8093EA00C091A500D091A600CE01DD
:1006A00004968F7799279093A6008093A500A3DFE7
:1006B0008091A5006091C9008F5F9DDF8091A500AA
:1006C0006091EA008E5F97DFCEBB84E18CBB86E150
:1006D0008CBBE199FECF8C2F8F5F8EBB84E18CBBEE
:1006E00086E18CBBE199FECF8C2F8E5F8EBB84E1BF
:1006F0008CBB86E18CBBE199FECFCD5FCEBB84E1A4
:100700008CBB86E18CBBE199FECF8091A5006DE5A5
:100710008D5FDF91CF916FCF1F920F920FB60F9227
:1007200011242F933F938F939F9384B195B1209180
:10073000AA00213039F49C013695279536952795E6
:100740002093AC002091AA002330E1F48D51914018
:100750002091AB002223A1F02091AB0030E02817BC
:10076000390728F42091AB002F5F2093AB00209134
:10077000AB0030E08217930728F48091AB008150E2
:100780008093AB008091AA008F5F8093AA00843091
:1007900010F01092AA008091AA00823010F481E833
:1007A00001C08FE887B99F918F913F912F910F9052
:1007B0000FBE0F901F9018951F920F920FB60F92B9
:1007C00011242F933F934F935F936F937F938F9356
:1007D0009F93AF93BF93EF93FF938091EB00882398
:1007E00021F081508093EB00E3C48091A8009091A8
:1007F000A900892B49F08091A8009091A900019748
:100800009093A9008093A800B7DE2091B7003091A3
:10081000B800892B09F4E4C1203D87E0380730F4A3
:100820002F5F3F4F3093B8002093B7008091B700FF
:100830009091B800823E24E0920791F42091C70085
:1008400021110EC01092C6001092E5001092BB005C
:100850001092C50081E08093C0001092BF00A8C430
:100860003091BF002091B0003323B1F01092BC0052
:1008700021119EC48332910521F48091BF008F5FC6
:1008800008C08634910509F093C481E08093B000DC
:100890008FE08093BF008CC4211197C12091C700C5
:1008A000222349F0019709F0AAC08091C00081116C
:1008B000A6C086E97AC02091CD00222309F49FC00A
:1008C000429708F49CC08091C000811198C080912B
:1008D000C100811194C08091BB00803508F08FC0A9
:1008E0001092A2008091C500813009F453C038F005
:1008F000823009F45DC0833009F464C080C0809107
:10090000C600811120C081E08093C50087E18093FB
:10091000E7008091F10089BD18BC8091E800882330
:1009200011F080E090DC8FEF8093C6008093E500AB
:100930008091C200811104C08091C6008093C200E2
:100940001092C3005CC08091C3009091C4008823C2
:1009500029F09093C5001092C30004C085E0891B64
:100960008093C5008091C6008F3FD9F08091C6006A
:10097000863940F083E08093C50086E98093E500E6
:1009800070DC3DC08091C6008130C9F582E0809363
:10099000C50035C08091E70081508093E700811148
:1009A0002EC082E08093C50081E08093C600E6CF30
:1009B0008093C4008091C6008639B0F48091C6004F
:1009C0008F5F09C08093C4008091C600823060F0C0
:1009D0008091C60081508093C6008093E50080918D
:1009E000C6008093C20008C084E08093C50080E008
:1009F0009ADC87E090E01EDC8091E50094DC809139
:100A0000CD00811135C08091B7009091B800489712
:100A100079F58091C00081112BC08091BB0080319D
:100A200090F48091C70081110EC08091CC00882382
:100A300011F0BBDD1DC08091BB00813011F410921C
:100A4000BB00C7DD15C08091BB008B3588F080915D
:100A5000F300811102C08091630081508093F30004
:100A6000E091F300F0E0EC56FF4F80818093BB00F3
:100A70008091B7009091B8008B34910509F072C055
:100A80008091B600823009F58091B3009091B40056
:100A90000E97D8F48091CD00882329F08091C00072
:100AA000813009F05FC01092C6001092E5001092EC
:100AB000BB001092C5009091C00081E0282F291B37
:100AC0002093C0008093C1004DC08091C00081116F
:100AD00049C08091B600813099F42091B3003091E3
:100AE000B4002E30310560F49091CD0091113AC0E0
:100AF00090E59093BB008093C10019BC18BC32C034
:100B00008091BB008B3510F054DC2CC08091BB0071
:100B1000803531F41092BB0019BC18BC85E109C0C6
:100B20008091BB00823569F41092BB0019BC18BCDF
:100B30008EE08093BF001092BD0081E08093B000F2
:100B400011C08091CD0081110DC08091E6008823F5
:100B500049F08091BB00803529F08091C700811158
:100B600001C01ADC8091C00081112FC08091C700A4
:100B700081112BC08091CD0081110FC08091B700F1
:100B80009091B800883C910541F48091B600823084
:100B900021F08091BB00803559F48091CD008823ED
:100BA000A1F08091B7009091B800843F914069F422
:100BB0001092BB001092C6001092C50019BC18BC60
:100BC00081E08093BF001092BD001092A1001092AE
:100BD000A00088E391E09093610080936000DEC202
:100BE0001092B0008091BF008823A1F0211531053B
:100BF00059F02831310528F48091BD008F5F809332
:100C0000BD001092BC00C6C28091BC008F5F809373
:100C1000BC00C0C2232B09F448C18091C7008823BF
:100C200031F01092C6001092E50080E07CDB20914C
:100C3000CD008091B7009091B800222309F487C0BD
:100C40001092C500429708F076C08091B6008F5F81
:100C50008093B6008091B600813009F075C0809114
:100C6000BB0080939F008091BB00803138F480915D
:100C7000C600863919F48FEF80939F008091BB00E6
:100C8000803541F08091BB00813521F08091BB001F
:100C9000823549F41092BB001092C6001092E50014
:100CA00081E08093C1008091C60080939E00809176
:100CB000C000811149C08091C100811145C080915F
:100CC000C700811141C08091C60081111FC0809171
:100CD000C200811103C081E08093C20081E0809353
:100CE000C30092E09093C4009091C2009093C6001C
:100CF0009093E5009091EC0091118093A70089EA10
:100D000093E09093A9008093A80004C01092C600BD
:100D10001092E5008091E5008F3F59F48091F10039
:100D200089BD18BC8091E800882371F080E08BDADF
:100D30000BC0F9DA09C01092B6008091EC0088234C
:100D400019F081E08093A7001092C100A9C08831FA
:100D5000910508F089C08091BB00803541F08091F9
:100D6000BB00813521F08091BB00823561F4809118
:100D7000BB0080939F001092BB008091B6008F5FF4
:100D80008093B6008DC08091BB00811106C0809118
:100D9000B600811102C081E007C08091B6008823AF
:100DA00029F08091B6008F5F8093B6008091C000DB
:100DB000811176C08091F000882399F08091B50070
:100DC000882379F08091BB0081110BC08091C7000E
:100DD000811166C08091B5008093BB001092B50070
:100DE0005FC08091BB00803110F58091C7008111F8
:100DF00057C08091BB00882391F08091B3009091FF
:100E0000B4008B34910558F08091BB008093B500FD
:100E10008091BB008093BA001092BB0041C08091CA
:100E2000CC00882311F0D5DB3BC0BFDB39C08091FB
:100E3000B3009091B4008B34910510F0BADA30C051
:100E40008091E6008130D1F3E091F300EF5FE09311
:100E5000F30080916300E81788F7F0E0EC56FF4F4D
:100E600080818093BB001CC08B349105B8F48091C5
:100E7000B600813099F42091B3003091B4002E3047
:100E8000310560F49091BB00911108C09091E80089
:100E9000891B8093E8008091E800D5D91092B600B4
:100EA0001092B4001092B30075C18091B30090917C
:100EB000B40001969093B4008093B300892B31F471
:100EC00080E395E79093B4008093B3008091B300E2
:100ED0009091B4000F9708F4A4C08091B6008530BB
:100EE000B9F48091CD00882309F499C08091C000A5
:100EF000811195C08091C700811191C081E08093DC
:100F0000C7001092C6001092E5001092BB0038C0D6
:100F10008091B6008430F9F48091CD00811105C034
:100F20008091C000882309F47AC08091C7008111A4
:100F300076C01092C6001092E5001092BB0010928D
:100F4000C5009091C00081E0282F291B2093C0008C
:100F50008093C10064C080919F0090EB980F923005
:100F600090F49091B600923009F059C0803511F498
:100F700081E501C082E58093BB0081E08093C100E0
:100F800019BC18BC4CC08091CD00882309F447C01F
:100F90008091C000811143C08091C70081113FC082
:100FA0008091B600833041F480E58093BB0081E0FE
:100FB0008093C10019BC18BC8091B600823079F5CD
:100FC00080919F008F3FC9F48091E600882311F043
:100FD000E3D925C08091C200863939F08091A20002
:100FE0008093C6008093E50004C01092C600109262
:100FF000E5008091E50097D912C086E98093C6008C
:101000008091C6008093E5008ED980919E008093E8
:10101000A20089EA93E09093A9008093A80010921F
:10102000B6008091CB008230E8F18091CD0088231A
:10103000E1F08091E50084578B38A0F58091A00005
:101040009091A10001969093A1008093A00020911F
:10105000B1003091B2002817390720F586E6809359
:10106000C6008093E500FDD81DC08091BB00803193
:10107000C8F4E091BB00F0E0E253FF4F80818F3F66
:1010800089F48091A0009091A10001969093A10015
:101090008093A0002091B1003091B2002817390749
:1010A00008F497DA8091CD00882391F08091C600F2
:1010B000823070F08091C600863950F48091B30080
:1010C0009091B4008C34910518F081E08093C300B6
:1010D0008091600090916100009729F001979093B2
:1010E0006100809360008091600090916100892B85
:1010F000D1F59091BB008091CD00811104C081E0B9
:10110000913041F408C09091E50081E0913019F0F0
:101110009F3F09F080E02091AC0030E0811103C0D6
:101120008BEA90E002C081EA90E02817390734F496
:1011300080919D008F5F80939D0004C010929D0060
:101140001092AE0080919D00883068F081E080931D
:10115000AF008093AE0010929D0088E391E09093E1
:101160006100809360008091AE00882399F08091A7
:101170009B0090919C00019690939C0080939B0013
:10118000843F914039F481E08093AD0010929C003F
:1011900010929B001092B8001092B70080919A00B4
:1011A0008F5F80939A00837019F486B1886486B942
:1011B000FF91EF91BF91AF919F918F917F916F912F
:1011C0005F914F913F912F910F900FBE0F901F9005
:1011D000189517BA88E088BB85BB83E087BB81EA96
:1011E0008ABD81E083BF81E887B9A29A87EC86B97E
:1011F000479A85B7877E806185BFF8948BB78F7DCE
:101200008BBFA89584B7877F84BF81B5886181BD76
:1012100011BC95D81092A6001092A5000091A500CF
:101220001091A6000038110508F028C5C8015ED548
:10123000F82E8093EE00C801019658D5D82F8093E0
:10124000C900C801029652D5C82F8093EA00C80190
:1012500003964CD58D3539F00C5F1F4F1093A600C7
:101260000093A500DBCF8F2D87708093BB008F2D5F
:101270008695869586958F708093ED00FF1CFF24E0
:10128000FF1CF092CD008D2F81708093CC00D1FB9C
:10129000882780F98093F0008D2F8695869587703A
:1012A0008093F100D295D695D770D093CB008C2F38
:1012B00081708093C800C1FB882780F98093EC007F
:1012C000C2FB882780F98093EF00C3FB882780F951
:1012D0008093E300C4FB882780F98093F200C295D5
:1012E000C695C370C093E6008091EF008093E8003C
:1012F0008AEF90E0FBD49FEF980F9E3F10F480930D
:101300006200C2D7E091CB00F0E0EE0FFF1FE45A7D
:10131000FF4F859194919093B2008093B10080919A
:10132000C800882359F08091CD00811107C08091B9
:10133000F400811105C039D967D902C01092BB00F1
:101340008091BB0081110CC08091CD00811104C03F
:101350008091C800811104C060E570E082E03BD854
:101360001092F4008AEF8093E90089E18093EB000A
:10137000F894A89581B5886181BD80E481BD789499
:10138000812C912C312CC1E0DFE058E2552E1FEF6B
:1013900068E3C62EDD24D3947CEFE72E7AE0F72EA7
:1013A000E5E0AE2EB12C44244A948091BF00811117
:1013B0008FC28091C0003816A9F03090C00019BCCF
:1013C00018BC6BE470E084E006D81092C1008091F4
:1013D000C000882329F08091BB008093E90002C0FF
:1013E0004092E9008091C700981669F09090C7007C
:1013F0006CE370E082E0EFD78AEF90E01BD76BE4FC
:1014000070E083E0E8D79091BB008091E9009817E5
:1014100009F409C18091BB00803140F52091BB00E7
:10142000822F90E0FC01E852FF4F30813093E400BE
:10143000FC01E253FF4F80818093CA008091CA0073
:101440009091E40099BD88BD211106C08091E8000B
:10145000882311F081E004C08091E900811101C06E
:10146000F2D68091BB008093E900DDC08091BB0083
:101470008093E90019BC18BC8091BB00803501F550
:1014800080E991E0D7D61092C1008091BB008035F1
:1014900009F0C9C080E09091AC00E82FF0E0E45D75
:1014A000FF4FE491E91710F48E5FF5CF8111825060
:1014B000E82FF0E0E35DFF4F849160E5DDD7E5CFF5
:1014C0008091BB00813579F48AEF90E0B3D6109219
:1014D000C1008091BB00813509F0A5C08091AB00AF
:1014E00061E5CAD7F6CF8091BB00823571F48AEFEF
:1014F00090E0A0D61092C1008091BB00823509F027
:1015000092C062E58CE0B8D7F7CF8091BB008B35F5
:1015100049F48091BB008B3509F085C069E28EE00B
:1015200029D7F7CF8091BB008C35E1F48091BB00C7
:101530008C3509F078C008E08091BB008C3511F043
:1015400008E00BC068E284E115D70150A9F7F8CF95
:1015500060E588E20FD7015049F38091BB008C35DC
:10156000B9F3E4CF8091BB008D3529F58091BB00A4
:101570008D35F1F404E08091BB008D3511F00AE067
:1015800012C019BC18BD85E090E054D619BD18BC36
:1015900081E490E04FD6015071F7F1CF88E490E0FC
:1015A00049D6015019F38091BB008D35B9F3DECFD8
:1015B00019BC18BC38C08091BB008E35C1F4809135
:1015C000BB008E3581F58CE291E034D66DE78DE776
:1015D000D1D66DE78DE7CED60FE08091BB008E357A
:1015E00071F784E690E026D60150B9F7E8CF8091F4
:1015F000BB008F35C1F48091BB008F35A1F48CE224
:1016000091E018D660EF80EFB5D660EF80EFB2D6EC
:1016100004E68091BB008F3571F784E690E00AD62E
:101620000150B9F7E8CF8091AF00882309F445C095
:101630008091CD00882369F18091E5008823D1F164
:10164000813011F08F3F61F487E08093E50088E0FE
:1016500034D71092C6001092E5001092C50012C057
:1016600083E02BD78091E5008A3050F090E0880F1E
:10167000991F880F991FB50112D36093E50002C02E
:10168000C093E5008091E5004ED68AEF90E0D2D578
:1016900011C08091BB00882369F08091BB0081302C
:1016A00011F488E001C083E008D78091BB0080314D
:1016B00008F48FD71092AF0034C08091AD0088231A
:1016C00081F18091EC00882351F18091E80088231A
:1016D000A9F08091CD00882321F08091E50081114F
:1016E00008C08091CD00811109C08091BB00882382
:1016F00029F062E084EF91E012D711C080E0A3D519
:1017000084EF91E097D581E09ED584EF91E092D56A
:1017100080E099D584EF91E08DD581E094D5109249
:10172000AD008091CB008130C9F59091AB008091E4
:101730006200981798F18091A8009091A900892BD8
:1017400069F58091CD008823C1F08091E5009EEB82
:10175000980F9D3B18F5282F30E066E094D2A90140
:10176000481B5109CA01423451050CF481E48093AD
:10177000E5008091E500D7D509C08091BB008823A2
:1017800069F08091BB00803148F423D7F092A90022
:10179000E092A80063E084EF91E0C1D68091AE00B2
:1017A000882329F034EE632E37E5732E04C026E338
:1017B000622E772473948091CD00811104C08091B2
:1017C000BB00882349F08091CD00882309F45AC0DA
:1017D0008091E500811156C0CFD6892B09F052C007
:1017E0008091B3009091B4006816790608F04AC061
:1017F0008091AC008B3A30F48091E800882311F09E
:1018000080E021D581E090E015D51092B4001092CF
:10181000B3001092A9001092A800F894A89584B77C
:10182000877F84BF81B5886181BD11BC789437986A
:101830001092B8001092B7009FD6892B21F080E15A
:1018400090E0F8D4F9CF8BB780628BBF85B7806208
:1018500085BF85B7846885BF8B7F85BF889585B731
:101860008F7D85BF8BB78F7D8BBF81E887B9A29AAB
:1018700087EC86B9F894A89581B5886181BD80E42C
:1018800081BD78948091A700882309F48ECD1092B1
:10189000A7008091E500882309F487CD82548D3B11
:1018A00010F402E001C001E08CE291E0C3D481E0D9
:1018B000CAD48FEA90E0BED480E0C5D4023029F4C7
:1018C0008FEA90E0B7D401E0F2CF0130E1F76DCDBF
:1018D0008091BD00881571F08090BD008091BD00A1
:1018E000882341F084E189BD18BC84E690E0A2D44D
:1018F00019BC18BC9091BF008091BE00981709F4E4
:10190000A1C18091BF008093BE001092BC00809165
:10191000BF00873109F47CC0E0F48E3009F448C080
:1019200028F4813059F1833091F1DFC08F3009F410
:101930005AC0853109F0D9C080E991E07BD481E0BB
:101940000AD68091BF008F5F8093BF001092BD00C8
:1019500076C1883209F473C138F4883109F467C05C
:10196000893109F471C0C1C0843609F479C0853663
:1019700009F481C0893209F0B8C08CC080E991E0D7
:1019800059D481E0E8D58091BF008F5F3AC1809142
:10199000BD00882359F08091BD00893038F48091D2
:1019A000BD0081708C278093CD002ED682E037C198
:1019B000C6D42AD68091EF008093E80065D48BE4EA
:1019C000809362006BE48AEF16D6E091CB00F0E0E2
:1019D000EE0FFF1FE45AFF4F859194919093B20050
:1019E0008093B1002AC11092BF0068E270E085E0E8
:1019F000F2D41092C6001092E5001092BB008091C4
:101A0000CD00882309F41BC18091C6008CD417C176
:101A10008091BD00882351F28091BD0081708C2798
:101A20008093EF008091EF008093E800BECF80911B
:101A3000BD00882339F08091BD0081708C27809390
:101A4000E300E2D583E0EBC08091BD00882309F478
:101A5000F4C08091BD0081708C278093EC00ECC0B5
:101A600068E270E083E0B7D419BC18BDD092A90039
:101A7000C092A800E4C019BC18BC8091A800909145
:101A8000A900892B11F56091AB00609362008AEF89
:101A9000B2D51BC08091BD008823B9F08091BD00F4
:101AA000873098F48091BD008F5F8093CB00ACD5D8
:101AB000E091CB00F0E0EE0FFF1FE45AFF4F85915D
:101AC00094919093B2008093B1008091CD008823CF
:101AD00021F084E040D585E003C088E03CD589E072
:101AE0008093BF008093BE00AAC08091CD00882360
:101AF000C1F18091BF008530A1F0863079F184304A
:101B000009F09DC08091BD00882309F49BCF80918E
:101B1000BD00883008F096CF8091BD008093F10021
:101B20003CC08091BD00813019F41092CB0013C0ED
:101B30008091BD00823009F460C08091BD00833087
:101B400059F466C0882341F08091BD0081708C27D4
:101B50008093F20099D358D584E061C08091BD0094
:101B600060C0E091BF008E2F90E0FC013497E73019
:101B7000F10508F064C0E15FFF4F8091BD0009945A
:101B8000882309F45FCF8091BD008D3008F05ACFD3
:101B90008091BD0081508093ED0076D352CF882391
:101BA00039F08091BD0081708C278093CC002CD5BA
:101BB00085E035C0882339F08091BD0081708C2785
:101BC0008093F00021D586E02AC0882351F08091CF
:101BD000BD00883030F48091BD008093F10054D373
:101BE00013D587E01CC0813021F41092CB000CD5B6
:101BF00015C08091BD00823039F4C093CB0004D56C
:101C000084E68093BF001BC08091BD00833031F417
:101C100068E270E0E0D35092BF0011C088E09BD42E
:101C20000EC0882351F08091BD00843030F4809143
:101C3000BD0081508093E600E7D4D093BF0010929E
:101C4000BD00B3CB8091BD00882321F08091BC0002
:101C50008E3770F48091BF00843609F4A6CB809152
:101C6000BD008111A2CB8091BC008C3D08F49DCBBE
:101C70008091BF008F5F8093BF0097CB1092A6002A
:101C80001092A50031CB991B79E004C0991F9617DB
:101C900008F0961B881F7A95C9F78095089597FBE1
:101CA000072E16F4009406D077FD08D00BD007FC61
:101CB00005D03EF4909581959F4F0895709561955C
:101CC0007F4F0895AA1BBB1B51E107C0AA1FBB1F72
:101CD000A617B70710F0A61BB70B881F991F5A95B8
:101CE000A9F780959095BC01CD010895E199FECFAB
:101CF0009FBB8EBBE09A99278DB30895F894FFCFD0
:101D000038014B05CE00CA00C400BC00B200A600DA
:101D1000980092008C00860080007800CF00CC00F4
:101D2000C700C000B700AC009F0095008F0089007D
:0A1D300083007C005B5C5D5E5F00D9
:00000001FF
